:100000000C942A000C9433141895000018950000E5
:10001000189500001895000018950000189500002C
:10002000189500000C949700189500001895000092
:10003000189500001895000018950000189500000C
:1000400018950000189500001895000018950000FC
:10005000189500008FE58DBFC0EDE8EC4E2E88E0CE
:100060008EBFD6E0F3E05F2EA89584B7082E877F79
:1000700084BF88E1992781BD91BDEEEFF7E0A0E64E
:10008000B0E088278D933197E9F780E189B980E066
:1000900080BD88E18AB9662487E886B980E487B99B
:1000A000D39AD29AD198B89AB99ABA9ABB9ABC9A6A
:1000B000A298A39AA49AA59AA69AA79A80E08FBD1F
:1000C00085E08EBD8F9A81E685BD74B7777F74BF5A
:1000D0008FE181BD87E081BD8B9885B78C7F826081
:1000E00085BFB59AB69A9A9AC99A839AA7EAB0E058
:1000F000E2E5FAE30E94F618A7EAB0E00E94E114F4
:1001000081E08093C7000091C700023018F011F021
:100110000C949700DA9A84E690E00E945515A7ECBB
:10012000B0E08C918F5F8C9310F40C94830070E09E
:1001300073BD789479B7746079BF85E08EBD379AC6
:1001400081B5886081BD7BB770647BBF00EE1DE424
:1001500020EE30E0ABEDB0E00D931D932D933C937A
:10016000ABEDB0E00D911D912D913C91ABEEB0E067
:100170000D931D932D933C93ABEEB0E00D911D912B
:100180002D913C91AFEEB0E00D931D932D933C93D8
:1001900000E011E020E030E0A3EDB0E00D931D930E
:1001A0002D933C93ABE4B1E0E6E0FAE30E94E8165D
:1001B00081E08093C7000091C700023018F011F071
:1001C0000C94F400DA9A82E390E00E945515DA98D4
:1001D00084E690E00E945515A7ECB0E08C918F5F0B
:1001E0008C9310F40C94DB000E942501AFEEB0E07C
:1001F0004D915D916D917C91ABEEB0E00D911D91B3
:100200002D913C910E94491B11F40C9409010E940C
:10021000C705A0EBB0E04D915C91AEEAB0E00D9166
:100220001C910417150711F40C9418010E949D06E7
:100230000E9417080E946C090E94D70881B5886146
:1002400081BD877F81BD0C94F40081E00E94C918B4
:1002500081E00E94C91882E00E94C91882E00E94D1
:10026000C91882E00E94C91887E00E94C91885E079
:100270000E94C9188AE00E94C91886E00E94C91825
:1002800085E00E94C91883E00E94C918E8E5FAE3F6
:100290000E94E714A0E6B0E088278C9381E0809369
:1002A000B2000091B200063218F011F00C948101F6
:1002B0000E94DB14A3EBB0E08C938FE3482F0091F6
:1002C000B300041711F00C946F010E94DB14A3EB30
:1002D000B0E08C9386E28093B2000C944601A3EBCD
:1002E000B0E08C91A0E6B0E00E94D4148D938827F2
:1002F0008C93A2EBB0E08C918F5F8C9310F40C94F4
:100300005101A3EDB0E08D919C919DBD8CBD81E02C
:10031000E0E6F0E002E00A93A0E9B0E00E94F21B00
:10032000A0E6B0E00E94321CEA2FFB2F32970FEFBD
:10033000A3E9B0E00E94F91BA0E9B0E0ECE5FAE324
:100340000E94381C81E009F480E08F93A3E9B0E0BB
:10035000E0E6FAE30E94381C81E009F480E09F9116
:10036000892B882311F40C94BE01DA98A881B981F5
:100370000E94E1140C9497000C94BF01DA9A85E076
:10038000E0E6F0E009E00A93A7E8B0E00E94F21B83
:10039000A7E8B0E00E94B51BABEDB0E00D931D9354
:1003A0002D933D93ABEDB0E00D911D912D913C91BE
:1003B000A7EFB0E00D931D932D933C9340E05BE3DA
:1003C00068E578E0ABEDB0E00D911D912D913C9189
:1003D0000E94491B0CF402C00C940302ABEDB0E088
:1003E0000D911D912D913C9144E050E060E070E052
:1003F0000E94D318ABEDB0E00D931D932D933D9368
:10040000AC980C942802ABEDB0E00D911D912D91AC
:100410003C9140E055E06AEE76E00E94441BABED73
:10042000B0E00D931D932D933D93ABEDB0E00D9196
:100430001D912D913C9144E050E060E070E00E94FD
:10044000D318ABEDB0E00D931D932D933D93AC9A73
:1004500082E1E0E6F0E006E00A93A5E9B0E00E9460
:10046000F21BA5E9B0E00E94B51BA7EDB0E00D932B
:100470001D932D933D93A7EDB0E00D911D912D910E
:100480003C9144E050E060E070E00E94D318A7ED9A
:10049000B0E00D931D932D933D9385E0E0E6F0E0F1
:1004A00004E00A93ACE9B0E00E94F21BACE9B0E0D2
:1004B0000E94B51BAEEAB0E00D931C938EE0E0E61F
:1004C000F0E004E00A93A0EAB0E00E94F21BA0EA88
:1004D000B0E00E94B51BAA89BB890C93AA89BB898D
:1004E0000C91003011F00C94810201E010E020E04A
:1004F00030E0AFEFB0E00D931D932D933C930C943F
:100500003F03013011F00C9491020AE010E020E06A
:1005100030E0AFEFB0E00D931D932D933C930C941E
:100520003F030A3011F00C94A10204E610E020E031
:1005300030E0AFEFB0E00D931D932D933C930C94FE
:100540003F030B3011F00C94B10208EE13E020E0F1
:1005500030E0AFEFB0E00D931D932D933C930C94DE
:100560003F030C3411F00C94C10208E213E220E0C6
:1005700030E0AFEFB0E00D931D932D933C930C94BE
:100580003F03043611F00C94D10200E117E220E0A1
:1005900030E0AFEFB0E00D931D932D933C930C949E
:1005A0003F03053611F00C94E10200EA16E821E061
:1005B00030E0AFEFB0E00D931D932D933C930C947E
:1005C0003F030E3611F00C94F10200E412E42FE028
:1005D00030E0AFEFB0E00D931D932D933C930C945E
:1005E0003F030F3611F00C94010300E816E928E9E7
:1005F00030E0AFEFB0E00D931D932D933C930C943E
:100600003F03083E11F00C94110302E310E020E0D8
:1006100030E0AFEFB0E00D931D932D933C930C941D
:100620003F03093E11F00C9421030AEF10E020E093
:1006300030E0AFEFB0E00D931D932D933C930C94FD
:100640003F03023F11F00C94310304EF11E020E06E
:1006500030E0AFEFB0E00D931D932D933C930C94DD
:100660003F03033F11F00C943F0308E813E120E03F
:1006700030E0AFEFB0E00D931D932D933C9388E1F4
:10068000E0E6F0E001E00A93AF85B8890E94F21B32
:10069000AE85BF850E94B51BABECB0E00C9389E141
:1006A000E0E6F0E001E00A93AD85BE850E94F21B12
:1006B000AC85BD850E94B51BACECB0E00C938DE120
:1006C000E0E6F0E001E00A93A989BA890E94F21BF2
:1006D000A889B9890E94B51BAAECB0E00C938EE101
:1006E000E0E6F0E001E00A93A5EAB0E00E94F21B28
:1006F000A5EAB0E00E94B51BA9ECB0E00C93A3E31F
:10070000B0E00C9102FB81E00EF080E08F9300914D
:10071000C800013081E009F480E09F91892388239B
:1007200011F40C94A30382E50E94EE1488E50E9464
:10073000EE148BE30E94EE14DB98C49881E0809362
:10074000C8000C94C503A3E3B0E00C9102FB81E068
:100750000EF480E08F930091C800013081E009F031
:1007600080E09F918923882311F40C94C50384E5CC
:100770000E94EE1488E50E94EE148BE30E94EE14B2
:10078000DB9AC49A80E08093C8000091CA000130CF
:1007900011F00C94CF03DB9AC49A0C94D103DB982C
:1007A000C4980091C900053081E009F080E08F9382
:1007B0000091C900043081E009F080E09F91892B0D
:1007C000882311F40C94E90381E08093CD000C940C
:1007D000EC0380E08093CD00A3E3B0E00C9102FB3A
:1007E00081E00EF480E08F930091CA00013081E037
:1007F00009F080E09F91892B882311F40C94A104C7
:10080000A3ECB0E08C918F5F8C930091C300053016
:1008100011F00C94730480E08093C300E2E6FAE3E5
:100820000E94E714AA85BB8588278C9381E080937A
:10083000B2000091B200063018F011F00C94490497
:100840000E94DB14A3EBB0E08C938FE3482F009160
:10085000B300041711F00C9437040E94DB14A3EBCF
:10086000B0E08C9386E08093B2000C94A204A3EBDA
:10087000B0E08C91AA85BB850E94D4148D93882703
:100880008C93A2EBB0E08C918F5F8C9310F40C945E
:100890001904A3EDB0E08D919C919DBD8CBD81E0CC
:1008A000EA85FB8504E00A93A985BA850E94F21BBC
:1008B000A885B985E8E6FAE30E94381C11F40C9487
:1008C00063040C94A20485E0EA85FB8501E00A93A9
:1008D000A985BA850E94F21BA885B9850E94B51B1F
:1008E000A6ECB0E00C930091C600003011F00C941F
:1008F0008404A8E3B0E08C9184FBA5E3B0E08C9184
:1009000085F98C930C94A2040091CA00013081E017
:1009100009F080E08F930091C600013081E009F07A
:1009200080E09F918923882311F40C949E0484E62F
:1009300090E00E945515AD9A0C949F04AD980C94CC
:10094000A204AD98A4ECB0E08C918F5F8C930091E1
:10095000C400053011F00C94B90580E08093C40008
:10096000EEE6FAE30E94E714AA81BB8188278C9304
:1009700081E08093B2000091B200043018F011F0D1
:100980000C94EB040E94DB14A3EBB0E08C938FE398
:10099000482F0091B300041711F00C94D9040E9461
:1009A000DB14A3EBB0E08C9384E08093B2000C9452
:1009B000B905A3EBB0E08C91AA81BB810E94D4144D
:1009C0008D9388278C93A2EBB0E08C918F5F8C93F2
:1009D00010F40C94BB04A3EDB0E08D919C919DBDEF
:1009E0008CBD81E0EA81FB8102E00A93A981BA8192
:1009F0000E94F21BA881B981E2E7FAE30E94381C49
:100A000011F40C9405050C94B90583E0EA81FB818F
:100A100001E00A93A981BA810E94F21BA881B981E1
:100A20000E94B51BAEECB0E00C930091CE000130FB
:100A300011F00C94B905A3E3B0E00C9102FB81E046
:100A40000EF080E08F930091CA00003081E009F041
:100A500080E09F918923882311F40C94B705E6E781
:100A6000FAE30E94E714AE81BF8188278C9381E06E
:100A70008093B2000091B200093018F011F00C948C
:100A80006A050E94DB14A3EBB0E08C938FE3482F40
:100A90000091B300041711F00C9458050E94DB1468
:100AA000A3EBB0E08C9389E08093B2000C94C10575
:100AB000A3EBB0E08C91AE81BF810E94D4148D93E2
:100AC00088278C93A2EBB0E08C918F5F8C9310F40D
:100AD0000C943A05A3EDB0E08D919C919DBD8CBD29
:100AE00081E0EE81FF8104E00A93AD81BE810E9426
:100AF000F21BAC81BD81EEE7FAE30E94381C11F4D1
:100B00000C9484050C94B90586E0EE81FF8103E026
:100B10000A93AD81BE810E94F21BAC81BD810E940F
:100B2000B51BAFECB0E00D931D932D933D934FEFAC
:100B300050E060E070E0AFECB0E00D911D912D91C0
:100B40003C910E94491B0CF002C00C94B1050FEFC0
:100B500010E020E030E0AFECB0E00D931D932D935A
:100B60003C93AFECB0E08C9183BD0C94B90570E080
:100B700073BD0091CE00003011F00C94C10570E0FF
:100B800073BD8CE2481A80E0580A66960895ABEE71
:100B9000B0E00D911D912D913C91AFEEB0E04D91E3
:100BA0005D916D917C910E94441BA3EFB0E00D9389
:100BB0001D932D933D93A3EFB0E00D911D912D91C9
:100BC0003C9144E050E060E070E00E94D318A3EF55
:100BD000B0E00D931D932D933D93A3EFB0E00D91E5
:100BE0001D912D913C91AFEFB0E04D915D916D91D4
:100BF0007C910E94D318A3EFB0E00D931D932D9329
:100C00003D93ABEDB0E00D911D912D913C91A3EF83
:100C1000B0E04D915D916D917C910E943F1BABEDD9
:100C2000B0E00D931D932D933D93ABEEB0E00D918D
:100C30001D912D913C91AFEEB0E00D931D932D933E
:100C40003C935A924A92ABEDB0E00D911D912D91DB
:100C50003C91D2010D931D932D933C9384E00E940F
:100C6000CF180E943806229684E00E94B614089598
:100C70008CE00E94C9188EE00E94C918AC81BD8129
:100C80000D911D912D913C9144E050E060E070E0A9
:100C90000E94F514AC81BD814D935D936D937D935E
:100CA000AC9B0C946706AC81BD810D911D912D917B
:100CB0003C9140E055E06AEE76E00E943F1BAC813B
:100CC000BD810D931D932D933D930C946706AA81CE
:100CD000BB81EC81FD810E945F1BEA81FB81A0EB5F
:100CE000B3E00E94E71BE0EBF3E0AA81BB81112790
:100CF00022270BE033270E94011BA881B981E4E879
:100D0000FAE30E94F618EA81FB81A881B9810E946A
:100D1000D4140E94E71BA881B9810E94D414E0E694
:100D2000FAE30E94F618A881B9810E94E1148AE1D1
:100D3000481A80E0580A24960895AEEAB0E00D9172
:100D40001C910A3050E015070CF402C00C94AC065C
:100D50000C949D060C940E08AEEAB0E00D911C9127
:100D60000A3050E0150780E00CF081E08F93AEEA86
:100D7000B0E00D911C910E3150E0150781E014F0A8
:100D800009F080E09F918923882311F40C94CC060C
:100D900076E078BB0C940E08AEEAB0E00D911C91A1
:100DA0000E3150E0150780E00CF081E08F93AEEA41
:100DB000B0E00D911C91023350E0150781E014F072
:100DC00009F080E09F918923882311F40C94EC06AC
:100DD00075E078BB0C940E08AEEAB0E00D911C9162
:100DE000023350E0150780E00CF081E08F93AEEA0B
:100DF000B0E00D911C91003550E0150781E014F032
:100E000009F080E09F918923882311F40C940C074A
:100E100074E078BB0C940E08AEEAB0E00D911C9122
:100E2000003550E0150780E00CF081E08F93AEEACA
:100E3000B0E00D911C91083750E0150781E014F0E7
:100E400009F080E09F918923882311F40C942C07EA
:100E500073E078BB0C940E08AEEAB0E00D911C91E3
:100E6000083750E0150780E00CF081E08F93AEEA80
:100E7000B0E00D911C91003A50E0150781E014F0AC
:100E800009F080E09F918923882311F40C944C078A
:100E900072E078BB0C940E08AEEAB0E00D911C91A4
:100EA000003A50E0150780E00CF081E08F93AEEA45
:100EB000B0E00D911C910E3B50E0150781E014F05D
:100EC00009F080E09F918923882311F40C946C072A
:100ED00071E078BB0C940E08AEEAB0E00D911C9165
:100EE0000E3B50E0150780E00CF081E08F93AEEAF6
:100EF000B0E00D911C910C3D50E0150781E014F01D
:100F000009F080E09F918923882311F40C948C07C9
:100F100070E078BB0C940E08AEEAB0E00D911C9125
:100F20000C3D50E0150780E00CF081E08F93AEEAB5
:100F3000B0E00D911C910E3051E0150781E014F0E6
:100F400009F080E09F918923882311F40C94AC0769
:100F500079E078BB0C940E08AEEAB0E00D911C91DC
:100F60000E3051E0150780E00CF081E08F93AEEA7F
:100F7000B0E00D911C91003951E0150781E014F0AB
:100F800009F080E09F918923882311F40C94CC0709
:100F900078E078BB0C940E08AEEAB0E00D911C919D
:100FA000003951E0150780E00CF081E08F93AEEA44
:100FB000B0E00D911C91063252E0150781E014F06B
:100FC00009F080E09F918923882311F40C94EC07A9
:100FD00077E078BB0C940E08AEEAB0E00D911C915E
:100FE000083755E0150780E00CF081E08F93AEEAFA
:100FF000B0E00D911C91043A56E0150781E014F021
:1010000009F080E09F918923882311F40C940C0847
:1010100078E078BB0C940E080C949D06AEEAB0E024
:101020008D919C91A0EBB0E08D939C93089587E007
:101030000E94C91885E00E94C91881E00E94C91861
:10104000A3E3B0E00C9102FB81E00EF080E08F930F
:101050000091CA00003081E009F080E09F9189236F
:10106000882311F40C94D108A2ECB0E08C918F5F2E
:101070008C930091C2000A3011F00C94CF0880E0EC
:101080008093C200E8E8FAE30E94E714AC81BD81D6
:1010900088278C9381E08093B2000091B2000630E3
:1010A00018F011F00C947D080E94DB14A3EBB0E063
:1010B0008C938FE3482F0091B300041711F00C9428
:1010C0006B080E94DB14A3EBB0E08C9386E0809366
:1010D000B2000C94D108A3EBB0E08C91AC81BD813F
:1010E0000E94D4148D9388278C93A2EBB0E08C914E
:1010F0008F5F8C9310F40C944D08A3EDB0E08D91AC
:101100009C919DBD8CBD81E0EC81FD8104E00A9342
:10111000AB81BC810E94F21BAA81BB81EEE8FAE39D
:101120000E94381C11F40C9499080C94D1080C946A
:10113000A90885E0EC81FD8101E00A93AB81BC81C7
:101140000E94F21BAA81BB810E94B51BA881B981B4
:101150000C93A881B9810C91003011F00C94B20865
:10116000AF9AAE98A881B9810C91013011F00C941E
:10117000BB08AF98AE98A881B9810C91023011F0EC
:101180000C94C408AF9AAE9AA881B9810C9103302F
:1011900011F00C94CD08AE9AAF980C94D1080C9431
:1011A000D1088DE0481A80E0580A2696089585E017
:1011B0000E94C91882E00E94C91881E00E94C918E3
:1011C000A3E3B0E00C9102FB81E00EF480E08F938A
:1011D0000091CA00013081E009F080E09F91892BE5
:1011E000882311F40C946509A5ECB0E08C918F5F15
:1011F0008C930091C500033011F00C94630980E0DA
:101200008093C500E4E9FAE30E94E714AC81BD8154
:1012100088278C9381E08093B2000091B200043063
:1012200018F011F00C943D090E94DB14A3EBB0E020
:101230008C938FE3482F0091B300041711F00C94A6
:101240002B090E94DB14A3EBB0E08C9384E0809325
:10125000B2000C946609A3EBB0E08C91AC81BD8127
:101260000E94D4148D9388278C93A2EBB0E08C91CC
:101270008F5F8C9310F40C940D09A3EDB0E08D9169
:101280009C919DBD8CBD83E0EC81FD8101E00A93C2
:10129000AB81BC810E94F21BAA81BB810E94B51B5D
:1012A000A881B9810C93A881B9810C91013011F00A
:1012B0000C945B09AB9AA881B9810C91003011F0B4
:1012C0000C946309AB980C946609AB9888E0481AB3
:1012D00080E0580A2696089584E00E94C91882E0AA
:1012E0000E94C91882E00E94C91882E00E94C918B1
:1012F00084E00E94C91884E00E94C91884E00E941A
:10130000C91884E00E94C91884E00E94C918A889FD
:10131000B989EEE0FAE30E94F91AA3E3B0E00C9178
:1013200002FB81E00EF480E08F930091CA0001304F
:1013300081E009F080E09F91892B882311F40C94BF
:10134000D70A07B1007E006007B90E94FC18AE857D
:10135000BF858D939C9307B1007E046007B90E94FE
:10136000FC18AC85BD858D939C93AE85BF854D9152
:101370005C91AC85BD850D911C910417150710F487
:101380000C94CE09AE85BF850D911C9141E050E0D3
:10139000041B150BAC85BD850D931C93EE85FF8555
:1013A000D190E080FF2400270E9499190E94C21961
:1013B0002F933F934F935F93EC85FD85D190E08011
:1013C000FF2400270E9499195F914F913F912F911F
:1013D0000E94DD19EDE0F0E0AA81BB810E94EC1BC8
:1013E000EA81FB810E947A19E2E1FAE30E94C61ABF
:1013F0000E94741AEDE0F0E0AA81BB810E94EC1B10
:10140000EE85FF85D190E080FF2400270E94991986
:101410000E94C2192F933F934F935F93EC85FD85F4
:10142000D190E080FF2400270E9499195F914F918D
:101430003F912F910E94DD19EDE0F0E0A881B98184
:101440000E94EC1BE881F9810E947A19E2E1FAE33B
:101450000E94C61A0E94651AEDE0F0E0A881B981E9
:101460000E94EC1BE881F9810E947A19EA81FB81D4
:101470000E9475190E94DD19EDE0F0E0AE81BF8198
:101480000E94EC1BEE81FF81AC81BD810E94EC1BB0
:10149000EE81FF810E947519EEE0FAE30E94CF1AF7
:1014A0000E94D81A18F011F00C94580A0C945E0A95
:1014B000AE81BF81EEE0FAE30E94F91AE889F9896A
:1014C0000E944D1C2D2D3E2D4F2D502FE6E1FAE3AD
:1014D0000E94C61A0E94DD19EDE0F0E0A885B985EA
:1014E0000E94EC1BEE81FF810E944D1C2D2D3E2D94
:1014F0004F2D502FE885F9850E9475190E94331AE7
:10150000EDE0F0E00E943719AA85BB85DD92EC92F0
:10151000AA85BB858C9183BDEE81FF810E947519E0
:10152000EAE1FAE30E94CF1A0E94D81A18F011F0EB
:101530000C949C0A0C94D70AEC81FD810E947519C9
:10154000EAE1FAE30E94CF1A0E94D81A80E010F074
:1015500009F081E08F93EE81FF810E947519EEE022
:10156000FAE30E94CF1A0E94D81A81E010F009F025
:1015700080E09F918923882311F40C94C30AE8E941
:10158000FAE30E94E714EC81FD810E947519EEE0F8
:10159000FAE30E94CF1A0E94D81A18F011F00C94A6
:1015A000D30A0C94D70AE0EAFAE30E94E7148EE12A
:1015B000481A80E0580A6296089581E00E94C9188E
:1015C00081E00E94C91884E00E94C918AC81BD81E5
:1015D000BA93AA935A924A9287E8D2018C9381E0F7
:1015E0000E94CF180E941414249681E00E94B61421
:1015F000AC81BD818C9181608C935A924A9287E82C
:10160000D2018C9381E00E94CF185A924A92A88509
:10161000B9858C91D2018C9381E00E94CF180E94F1
:101620000214249682E00E94B61481E0AC81BD8150
:101630008C93AC81BD810C91003011F40C94390B6A
:10164000AC81BD81BA93AA935A924A9287E8D2019B
:101650008C9381E00E94CF180E941414249681E09C
:101660000E94B614AC81BD818C9181708C930C94D6
:10167000190B81E08093B4000091B400063018F09B
:1016800011F00C946B0B0091B40046E0040FA5EB35
:10169000B0E00C93A4EBB0E0AD90BB24A5EBB0E0C0
:1016A000AA0DBB1DBA93AA935A924A928091B50093
:1016B000D2018C9381E00E94CF180E9414142496CA
:1016C00081E00E94B614A4EBB0E08C918F5F8C9304
:1016D00010F40C943C0BA6EBB0E00C9111272227E0
:1016E000332740EE50E060E070E00E944915A3EE21
:1016F000B0E00D931D932D933D9395E0A3EEB0E0E4
:101700000E942619A3EEB0E00D911D912D913C9100
:1017100044E050E060E070E00E943F1BA3EEB0E0C8
:101720000D931D932D933D930091B6004FE104233B
:10173000AC81BD810C9392E0AC81BD810E94051902
:101740000091B70040EC0423AA81BB810C9396E082
:10175000AA81BB810E941E19AC81BD810C91112709
:1017600022273327AA81BB814C91552766277727EB
:101770000E943F1BA7EEB0E00D931D932D933D9368
:1017800040E050E060E070E0A7EEB0E00D911D9108
:101790002D913C910E94491B11F00C94DB0B01E050
:1017A00010E020E030E0A7EEB0E00D931D932D9304
:1017B0003C930C94FB0B0091E70041E00423AC81C7
:1017C000BD810C93AC81BD810C91003011F40C945F
:1017D000FB0BA7EEB0E00D911D912D913C9141E0E6
:1017E00050E060E070E00E943F1BA7EEB0E00D9378
:1017F0001D932D933D93A7EBB0E00C911127222769
:1018000033274FE350E060E070E00E944915A88163
:10181000B9810D931D932D933D9394E0A881B981D7
:101820000E940D190091B80040EF0423AC81BD81E6
:101830000C9394E0AC81BD810E941E19A881B981EE
:101840000D911D912D913C91AC81BD814C915527FD
:10185000662777270E943F1BA881B9810D931D93AE
:101860002D933D93A881B981E3E2F1E00E94321803
:10187000A8EBB0E00C911127222733274FE050E06E
:1018800060E070E00E944915A881B9810D931D9315
:101890002D933D9398E0A881B9810E940D19A881EC
:1018A000B9810D911D912D913C91A9EBB0E04C9126
:1018B0005527662777270E943F1BA881B9810D9382
:1018C0001D932D933D9398E0A881B9810E940D1935
:1018D000A881B9810D911D912D913C91AAEBB0E0A9
:1018E0004C915527662777270E943F1BA881B98115
:1018F0000D931D932D933D9398E0A881B9810E948B
:101900000D19A881B9810D911D912D913C91ABEBE1
:10191000B0E04C915527662777270E943F1BA8818E
:10192000B9810D931D932D933D93A881B981EBE26D
:10193000F1E00E943218ABE2B1E0BA93AA93EEE173
:10194000FAE3ABE1B1E00E94E816EBE2F1E00E94BD
:101950001F162296ABE2B1E0BA93AA93ABE2B1E0D4
:10196000E3E2F1E00E9478152296A3EEB0E0E3E214
:10197000F1E00E943218A3E3B1E0BA93AA93E6E241
:10198000FAE3ABE1B1E00E94E816EBE1F1E0A3E29B
:10199000B1E00E94B3152296A7EEB0E0E3E2F1E0D9
:1019A0000E943218A3E3B1E0BA93AA93A3E2B1E094
:1019B000E3E3F1E00E94B3152296A3E3B1E0BA930A
:1019C000AA93ABE2B1E0E3E3F1E00E941F16229696
:1019D000E3E3F1E0ABE3B1E00E940717A3E4B1E079
:1019E000E0E0F0E098E00E941B1CA3E4B1E0EEE22E
:1019F000FAE30E94C11680E010F009F081E08F93B5
:101A0000A3E4B1E0E6E3FAE30E94C11681E008F046
:101A100080E09F91892B882311F40C94170DA3E388
:101A2000B1E0EEE3FAE30E94E8160C941D0DE3E446
:101A3000F1E0A3E3B1E00E94071786E0481A80E0D6
:101A4000580A2696089584E00E94C91884E00E94EE
:101A5000C91884E00E94C91884E00E94C9189AE05D
:101A6000A885B9850E94261905E51DE724E530E023
:101A7000A885B9854D915D916D917C910E94F51479
:101A8000AC81BD814D935D936D937D9308E415E426
:101A900028E430E0A885B9854D915D916D917C91E8
:101AA0000E94F514AE81BF814D935D936D937D933C
:101AB00092E0AC81BD810E942619AC81BD810C9160
:101AC00042E00E94221CA5EBB0E08C930091B5008F
:101AD000013011F00C947E0DAC81BD810D911D91F2
:101AE0002D913C9141E050E060E070E00E943F1B8E
:101AF000AC81BD810D931D932D933D93AE81BF812C
:101B00000D911D912D913C914BE050E060E070E013
:101B10000E94F514AE81BF814D935D936D937D93CB
:101B2000AE81BF810C9142E00E94221CA5EBB0E087
:101B30008C930091B500013011F00C94B10DAE8181
:101B4000BF810D911D912D913C9141E050E060E0ED
:101B500070E00E94441BAE81BF810D931D932D93B5
:101B60003D93AE81BF810D911D912D913C9141E03E
:101B700050E060E070E00E943F1BAE81BF810D939A
:101B80001D932D933D9340E850E060E070E0AC8100
:101B9000BD810D911D912D913C910E94491B1CF01E
:101BA00011F00C94D50D0C94DF0D00E810E020E04E
:101BB00030E0AC81BD810D931D932D933C9340E0AB
:101BC00050E060E070E0AE81BF810D911D912D91DC
:101BD0003C910E94491B1CF011F00C94F90D01E09E
:101BE00010E020E030E0AE81BF810D931D932D9376
:101BF0003C9300E010E020E030E0A881B9810D9333
:101C00001D932D933C9381E08093B4000091B40028
:101C1000063018F011F00C94D40EA885B9850D91FA
:101C20001D912D913C91A4EBB0E0AD90BB24ABEBAA
:101C3000B0E0AA0DBB1D4C915527662777270E945F
:101C4000D318AA81BB810D931D932D933D93AA8137
:101C5000BB810D911D912D913C91AC81BD814D9128
:101C60005D916D917C910E94D318AA81BB810D93E7
:101C70001D932D933D9348E455E468E470E0AA81F8
:101C8000BB810D911D912D913C910E94491B0CF03F
:101C900002C00C94CC0E45E55DE764E570E0AA81D6
:101CA000BB810D911D912D913C910E94491B1CF00F
:101CB00011F00C94CC0E40E050E060E070E0A881A0
:101CC000B9810D911D912D913C910E94491B11F0FC
:101CD0000C94920EAA81BB810D911D912D913C9186
:101CE000A881B9810D931D932D933C93A4EBB0E093
:101CF000AD90BB24ABEBB0E0AA0DBB1D8C91A3EE65
:101D0000B0E08D9388278D938D938C93AC81BD81AA
:101D10000D911D912D913C91A7EEB0E00D931D9377
:101D20002D933C93A881B9814D915D916D917C91EA
:101D3000AA81BB810D911D912D913C910E94491B5F
:101D40001CF011F00C94CC0EAA81BB810D911D9159
:101D50002D913C91A881B9810D931D932D933C93B6
:101D6000A4EBB0E0AD90BB24ABEBB0E0AA0DBB1D83
:101D70008C91A3EEB0E08D9388278D938D938C93F7
:101D8000AC81BD810D911D912D913C91A7EEB0E0EC
:101D90000D931D932D933C93A4EBB0E08C918F5F3A
:101DA0008C9310F40C94060EAC81BD810D911D91A5
:101DB0002D913C9142E050E060E070E00E94441BB5
:101DC000AC81BD810D931D932D933D93AE81BF8159
:101DD0004D915D916D917C91AC81BD810D911D9175
:101DE0002D913C910E94491B1CF011F00C94030EA4
:101DF00080E1481A80E0580A2896089584E00E94FD
:101E0000C91884E00E94C91884E00E94C91881E0C2
:101E10000E94C91881E00E94C91881E00E94C91877
:101E200081E00E94C91881E00E94C91888E00E94E0
:101E3000C91884E00E94C91884E00E94C918009162
:101E4000CA00003081E009F080E08F930091CB0060
:101E5000003081E009F080E09F9189238F93009109
:101E6000CC00003081E009F080E09F918923882335
:101E700011F40C944D0FABEDB0E00D911D912D912F
:101E80003C9140EA5CE860E070E00E94441BAE894F
:101E9000BF890D931D932D933D930091CA0000308F
:101EA00081E009F080E08F930091CB00003081E069
:101EB00009F080E09F9189238F930091CC0001303D
:101EC00081E009F080E09F918923882311F40C942C
:101ED0007B0FABEDB0E00D911D912D913C9140EA4F
:101EE0005CE860E070E00E94441BAE89BF890D93FE
:101EF0001D932D933D930091CA00003081E009F0BD
:101F000080E08F930091CB00013081E009F080E008
:101F10009F9189238F930091CC00013081E009F0DB
:101F200080E09F918923882311F40C94BD0FABEDC1
:101F3000B0E00D911D912D913C9140EA5CE860E08C
:101F400070E00E94441BAE89BF890D931D932D93B1
:101F50003D93AE89BF890D911D912D913C91A7EDC7
:101F6000B0E04D915D916D917C910E943F1BAE89D7
:101F7000BF890D931D932D933D930091CA000030AE
:101F800081E009F080E08F930091CB00013081E087
:101F900009F080E09F9189238F930091CC0000305D
:101FA00081E009F080E09F918923882311F40C944B
:101FB000FF0FABEDB0E00D911D912D913C9140EAEA
:101FC0005CE860E070E00E94441BAE89BF890D931D
:101FD0001D932D933D93AE89BF890D911D912D9138
:101FE0003C91A7EDB0E04D915D916D917C910E9487
:101FF0003F1BAE89BF890D931D932D933D93009197
:10200000CA00013081E009F080E08F930091CB009D
:10201000003081E009F080E09F9189238F93009147
:10202000CC00003081E009F080E09F918923882373
:1020300011F40C942710ABEDB0E00D911D912D9192
:102040003C91AE89BF890D931D932D933C930091D4
:10205000CA00013081E009F080E08F930091CB004D
:10206000013081E009F080E09F9189238F930091F6
:10207000CC00003081E009F080E09F918923882323
:1020800011F40C944F10ABEDB0E00D911D912D911A
:102090003C91AE89BF890D931D932D933C93009184
:1020A000CA00013081E009F080E08F930091CB00FD
:1020B000013081E009F080E09F9189238F930091A6
:1020C000CC00013081E009F080E09F9189238823D2
:1020D00011F40C947F10ABEDB0E00D911D912D919A
:1020E0003C91A7EDB0E04D915D916D917C910E9486
:1020F0003F1BAE89BF890D931D932D933D93009196
:10210000CA00013081E009F080E08F930091CB009C
:10211000003081E009F080E09F9189238F93009146
:10212000CC00013081E009F080E09F918923882371
:1021300011F40C94AF10ABEDB0E00D911D912D9109
:102140003C91A7EDB0E04D915D916D917C910E9425
:102150003F1BAE89BF890D931D932D933D93009135
:10216000CD00013081E009F080E08F930091CA003A
:10217000013081E009F080E09F918923882311F4E8
:102180000C94D410AE89BF890D911D912D913C9175
:1021900040EE5BEA60E070E00E94441BAE89BF89BC
:1021A0000D931D932D933D935A924A92A88DB98D0C
:1021B0000D911D912D913C91D2010D931D932D9365
:1021C0003C9384E00E94CF180E94230D229684E065
:1021D0000E94B614A3EEB0E0E3E2F1E00E943218F0
:1021E000AE89BF89EC81FD810E943218ABE2B1E07B
:1021F000BA93AA93AE81BF81E3E2F1E00E94B315E6
:102200002296A7EEB0E0E3E2F1E00E943218ABE2E2
:10221000B1E0BA93AA93A3E2B1E0EBE2F1E00E944D
:10222000B3152296C9990C943D11ABE4B1E0BA9371
:10223000AA93E6E4FAE3ABE1B1E00E94E816EBE42E
:10224000F1E00E94B3152296A3E3B1E0BA93AA93FA
:10225000ABE4B1E0E3E3F1E00E9478152296ABE451
:10226000B1E0E6E0FAE30E94E816E0E0F0E0A3E384
:10227000B1E098E07BE70E940A1CABE2B1E0BA93C0
:10228000AA93A3E3B1E0EBE2F1E00E941F162296CD
:1022900081E08093B4000091B400063018F011F092
:1022A0000C94641180E0A4EBB0E0AD90BB24A5EBEE
:1022B000B0E0AA0DBB1D8C93A4EBB0E08C918F5FB6
:1022C0008C9310F40C944B11A3EEB0E00D911D9182
:1022D0002D913C9144E050E060E070E00E94441B8E
:1022E000A3EEB0E00D931D932D933D9395E0A3EEE7
:1022F000B0E00E940D198091E3008093B60041E0A8
:1023000050E060E070E0A7EEB0E00D911D912D91DE
:102310003C910E94491B11F00C949A1100E010E0CE
:1023200020E030E0A7EEB0E00D931D932D933C9399
:102330000C94BA110091E70041E00423AC85BD85FF
:102340000C93AC85BD850C91003011F00C94BA1142
:10235000A7EEB0E00D911D912D913C9141E050E030
:1023600060E070E00E94441BA7EEB0E00D931D9367
:102370002D933D930091B60040EE0423AA85BB85C2
:102380000C938091E700A885B9858C9392E0A8858D
:10239000B9850E941E19AA85BB850C91A885B985AF
:1023A0004C91042BA6EBB0E00C930091E70043E0C6
:1023B0000423AE81BF810C9396E0AE81BF810E9461
:1023C0000519AE81BF818C918093B700EBE2F1E0FB
:1023D000A3E2B1E00E946A16AC81BD81BA93AA93D0
:1023E000A3E2B1E0EBE2F1E00E9463152296EC81FA
:1023F000FD81AA81BB810E94501894E0AA81BB8113
:102400000E942619AA81BB810C914FE30423AE855B
:10241000BF850C930091B700AE85BF854C91042B0E
:10242000A7EBB0E00C93A3E2B1E0BA93AA93EEE17C
:10243000FAE3ABE1B1E00E94E816E3E2F1E00E94CA
:10244000B3152296E3E2F1E0A881B9810E94501809
:10245000A881B9810D911D912D913C91AC89BD89C7
:102460000D931D932D933C9398E1AC89BD890E94F7
:102470002619AC89BD890C914FEF0423A8EBB0E07D
:102480000C93EC81FD81AA81BB810E94501894E0DD
:10249000AA81BB810E940D190091B800AA81BB815D
:1024A0004C91042BA8EBB0E00C93A881B9810D915D
:1024B0001D912D913C91AA89BB890D931D932D935C
:1024C0003C9390E1AA89BB890E942619AA89BB89FD
:1024D0000C914FEF0423A9EBB0E00C93A881B981D4
:1024E0000D911D912D913C91A889B9890D931D9352
:1024F0002D933C9398E0A889B9890E942619A88950
:10250000B9890C914FEF0423AAEBB0E00C93A8819A
:10251000B9810C914FEF0423ABEBB0E00C93AE8587
:10252000BF85BA93AA935A924A9289E8D2018C93B2
:1025300081E00E94CF180E941414249681E00E942A
:10254000B614AE85BF858C9180618C935A924A9265
:1025500089E8D2018C9381E00E94CF185A924A9266
:10256000AA89BB898C91D2018C9381E00E94CF18FB
:102570000E940214249682E00E94B61481E08093A7
:10258000B4000091B400063018F011F00C94F6126B
:102590000091B40046E0040FA5EBB0E00C935A9212
:1025A0004A928091B500D2018C9381E00E94CF18AD
:1025B0005A924A92A4EBB0E0AD90BB24A5EBB0E0F8
:1025C000AA0DBB1D8C91D2018C9381E00E94CF1883
:1025D0000E940214249682E00E94B614A4EBB0E09C
:1025E0008C918F5F8C9310F40C94C112AE85BF85D3
:1025F000BA93AA935A924A9289E8D2018C9381E0C5
:102600000E94CF180E941414249681E00E94B614F0
:10261000AE85BF858C918F7E8C935A924A9289E8C1
:10262000D2018C9381E00E94CF185A924A92AA89D3
:10263000BB898C91D2018C9381E00E94CF180E94BB
:102640000214249682E00E94B614AE85BF85BA9328
:10265000AA935A924A9287E8D2018C9381E00E9411
:10266000CF180E941414249681E00E94B614AE85FF
:10267000BF858C9180648C93A7E0B1E04D915D9112
:102680006D917C91A7EFB0E00D911D912D913C9142
:102690000E94491B80E00CF081E08F93ABE0B1E039
:1026A0004D915D916D917C91A7EFB0E00D911D91E1
:1026B0002D913C910E94491B81E014F009F080E0CB
:1026C0009F91892B882311F40C94FC13A7EFB0E0A1
:1026D0000D911D912D913C91A3E0B1E00D931D93BF
:1026E0002D933C93E7EFF0E00E9475190E94991931
:1026F000AFE0B1E00E94BD19EEE4FAE30E94CF1A08
:10270000EFE0F1E00E9475190E94331AEDE0F0E06D
:10271000AFE0B1E00E94EC1BEFE0F1E00E9437195E
:10272000A3E1B1E0EDE0FF270E94EC1BA3E0B1E0E4
:102730000D911D912D913C91A3E1B1E04D915D91E1
:102740006D917C910E943F1BA7E0B1E00D931D931A
:102750002D933D93A3E0B1E00D911D912D913C91FE
:10276000A3E1B1E04D915D916D917C910E94441B7C
:10277000ABE0B1E00D931D932D933D935A924A9295
:1027800087E8D2018C9381E00E94CF185A924A9236
:10279000AA89BB898C91D2018C9381E00E94CF18C9
:1027A0000E940214249682E00E94B61481E0AE8555
:1027B000BF858C93AE85BF850C91003011F40C94CD
:1027C000FA13AE85BF85BA93AA935A924A9287E8C4
:1027D000D2018C9381E00E94CF180E941414249699
:1027E00081E00E94B614AE85BF858C9180748C9375
:1027F0000C94DA130C94FC1381E2481A80E0580A16
:10280000669608950E94B11C1AEA0E94C91CAA810A
:10281000BB811C910E94C91CA881B9811C910E9496
:10282000C91C0E94C01C089580E0809353010E943F
:10283000B11C1AEA0E94C91CA881B9811C910E948E
:10284000C91C0E94B11C1BEA0E94C91C0E94E61C04
:10285000A3E5B1E01C930E94C01C80915301AA81A2
:10286000BB818C9308950F921F922F923F924F92AB
:102870005F927F92AF92BF920F931F932F933F93DC
:102880004F935F936F937F938F939F93AF93BF9378
:10289000CF93DF93EF93FF938FB78F93C99B0C94E4
:1028A000601483990C945A14ABEEB0E00E94BA14F1
:1028B0000C945E14ABEEB0E00E94C7140C946F143D
:1028C00083990C946B14ABE4B1E0ABE4B1E00E94EB
:1028D0009F160C946F14ABE4B1E00E94A21670E452
:1028E0007ABF8F918FBFFF91EF91DF91CF91BF9111
:1028F000AF919F918F917F916F915F914F913F9198
:102900002F911F910F91BF90AF907F905F904F904C
:102910003F902F901F900F90189504050607090B04
:1029200081E08093C7000091C700023018F011F0D9
:102930000C94AC14DA9A82E390E00E945515DA9870
:1029400082E390E00E945515A7ECB0E08C918F5F78
:102950008C9310F40C94931471E073BDE8E5FAE3E2
:102960000E94E7140895481A590A0895481A8827BA
:10297000580A08950D911D912D913C910F5F1F4FA5
:102980002F4F3F4F3C932E931E930E9308950D911E
:102990001D912D913C9101501040204030403C93BE
:1029A0002E931E930E9308958F938D918823E9F7AC
:1029B00011978F9108955F9BFECF8CB10895A0EB86
:1029C000B3E08D91882311F009D0FBCF08950E94C8
:1029D000C21A802D11F002D0FACF08955D9BFECF70
:1029E0008CB9089500FC05D0089530D005D001F8C9
:1029F000F9CF37D03FD00895842F952FA62FB72F2A
:102A0000E894452B462B472B11F468940895402FEA
:102A1000512F622F732F0027112722273327F0E22F
:102A2000440F551F661F771F001F111F221F331FE2
:102A3000081B190B2A0B3B0B416028F4080F191FC8
:102A40002A1F3B1F4E7FFA9559F708950024E894FA
:102A500077FF02C006D0689400F809D010F801246E
:102A6000089512D04F5F5F4F6F4F7F4F0895E894E6
:102A700037FF089500951095209530950F5F1F4FF3
:102A80002F4F3F4F689408954095509560957095ED
:102A90000895042315232623372308950895689461
:102AA00062F80895E89462F80895EF93FF93EE2793
:102AB000E82BE92B11F0E0EAFFE0FF91EF91089598
:102AC0007CD204D09EC10F0101D09EC1FD01FF93B5
:102AD000EF9387818F9390E889278783F0010BD04C
:102AE0008F91EF91FF918783089567D204D089C1B8
:102AF0000F0101D089C100E077D209F008959A0151
:102B0000281B390B1AF4D0010F01F5CF002727330A
:102B1000300708F09CC2822FA7D1BBD1C9D1372F73
:102B200036270AF4EDD1F0018081A80E8181B81E0C
:102B30008281C81E8381D81E8481E81E8581F81E8B
:102B400086818F708061081F1AF4DAD180E86827C7
:102B500005FF02C081E0AAD104FD01C004D2C2C1B8
:102B60002CD204D04EC10F0101D04EC108E13CD29D
:102B700009F00895480F591F4F5F534067276F931F
:102B80005F934F9320D22227F00179D193E0110F68
:102B9000331F441F551F661F771F881F9A95B9F76B
:102BA000FD01A7E0BB279191A13011F49F709061C6
:102BB000992301F1939FA00CB11CBB1F959FB69563
:102BC000C01CD11CBB1F979FB695E01CF11C0B1FAE
:102BD000919F200DA11CBB1F949FB695B01CC11CDA
:102BE000BB1F969FB695D01CE11CBB1F989FB69546
:102BF000F01C011DAA9549F02A2DAB2CBC2CCD2C24
:102C0000DE2CEF2CF02E0027CECF4F915F916F91ED
:102C100004FB16F05ED102C04F5F5F4F63C1FF93AC
:102C200009901124F8E0069408F4190E17940794FB
:102C3000FA95D1F7FF910895C0D104D0E2C00F01F9
:102C400001D0E2C004E2D0D109F00895481B590B2D
:102C500041505C4F67276F935F934F93F00104D10E
:102C60002FEFFD010CD1ADE3BA2FB77019F4209509
:102C70002F932FEFA116B306C406D506E606F70676
:102C8000080738F0A11AB30AC40AD50AE60AF70AF7
:102C9000080B221FAA0CBB1CCC1CDD1CEE1CFF1C4D
:102CA000001FAA9509F72095AF90BF90CF90DF90B5
:102CB000EF90FF900F914F915F916F9104FB1EF089
:102CC00008D1415050400EC1E881F981AA81BB81F1
:102CD0000895FADF02D0FD0182C0A1D0C5D0AC01B9
:102CE000632F61FD70C160FD6EC162FD77C14E5FF3
:102CF000534022F119F15523A9F7463398F748308C
:102D000048F00F2DFE2CED2CDC2CCB2CBA2CAA2459
:102D10004850A8F7413048F0AA0CBB1CCC1CDD1C65
:102D2000EE1CFF1C001F4150A9F7702F707E0F7121
:102D30004EEF53E018D135D1A9F2FBC059C0E8E2FB
:102D4000F1E303C0E8E2F1E30DC05D01FF93EF930F
:102D500007D2EF91FF913CD0F501FA93EA93C8DED8
:102D600022960CC25D01FF93EF93FAD1EF91FF9190
:102D70002FD0F501FA93EA93A6DE2296FFC1A8812F
:102D8000B981661778E06FB78D9195917A9599F032
:102D90006FBF89076FB7F8CFE881F981AA81BB813E
:102DA000661778E06FB78D9191917A9521F06FBF9A
:102DB00089076FB7F8CF70E8872797276FBF890714
:102DC00031F06FB7892B12F071E067276FBF08955C
:102DD00088E005900D928A95E1F718970895A082F2
:102DE000B182C282D382E482F5820683178308957A
:102DF000A080B180C280D380E480F58006811781F5
:102E00000895EC81FD81EBCFE881F981E8CF88E07E
:102E100091919D938A95E1F7189738970895868147
:102E20009781332797FB37F988949F7721F488237C
:102E300011F4326008952FEE28172FE7290740F488
:102E40002FE02823089411F4316008953460089528
:102E5000807F969587959695879596958795969573
:102E60008795989488940895A080B180C280D3807B
:102E7000E480F58006810F7000612227089510819B
:102E80003181428153816481758186818F70806137
:102E90000895883050F02A2DAB2CBC2CCD2CDE2C84
:102EA000EF2CF02E00278850F4CF0895689401C0CD
:102EB000E894882369F00595F794E794D794C7942C
:102EC000B794A794279516F44F5F5F4F8A95F1CF7B
:102ED0000895220FAA1CBB1CCC1CDD1CEE1CFF1C81
:102EE000001F089501D025C0203848F011F4A0FE3D
:102EF00006C0089412D005FF089581E0D7CF089549
:102F00002095A094B094C094D094E094F09400954F
:102F10000F9200240894201D0F9050F40F9200246B
:102F2000A01CB01CC01CD01CE01CF01C001D0F908D
:102F300008955523B2F0352F342B99F03FEF431706
:102F400037E0530778F4440F551F440F551F440FC3
:102F5000551F440F551F0F7E042B152F67FB17F9C4
:102F6000089531C037C087E03F2D303230E003078D
:102F700078F40F2DFE2CED2CDC2CCB2CBA2CA22EB1
:102F80002227485050408A9579F7442755271BC07F
:102F900088E004FD05C09DDF415050408A95C9F787
:102FA00008950F9200240A280B280C280D280E28BB
:102FB0000F28002A00200F900895EA81FB81A88144
:102FC000B9810F010895AA24BB246501750185010B
:102FD00098940895F8DF00EF1FE708958FEFA82E6B
:102FE000B82EF3DF1F7708951ADF632FAC01FD01C0
:102FF00016DF732F00C0372F362B3F7709F4089563
:1030000032FDECCF262F2727372F60FB32F961FBEB
:1030100033F93F70E0E3F1E3002311F427FD3C9620
:10302000030FE00F0027F01F849187FDD7CF86FDA7
:10303000D1DF85FDC8DF84FD0AD083FD0AD082FD83
:103040000AD081FD0BD080FD0BD098940895F0013B
:10305000CFCEFD01CDCE67FB17F9089577FBFCCFEE
:1030600027FBFACFCD90DD90ED90FD90AA24BB24F4
:103070000027112722276627FF2012F406D0606858
:1030800043E254E070DF55DFAACEC094D094E094C0
:10309000F09481E0C80E8827D81EE81EF81E089517
:1030A000BEDE31FD19C032FD17C030FD2AC08E5F73
:1030B000934092F0992329F5803238F4D5DE81953A
:1030C0008B5DE7DEE894F4DE0CC0CC24C094DC2CED
:1030D000EC2CFC2CF69412C0CC24DD24EE24FF242E
:1030E00010C080E8B81650F031F4BA28B22AB816E9
:1030F00011F4C0FC03C0CDDFF7FCE7CF37FF01C000
:10310000C4DFCD92DD92ED92FD920895B7FE089551
:1031100090E8B91611F4D0FE08959FEFD91AE90A84
:10312000F90A09F403950895000000000000F03F3B
:1031300000081000101010000808200000081000FF
:10314000108010000808200000412000414180004C
:103150002080200000204400418044002020800086
:1031600088E00FB6F8945A924A92E42DF52DA42DDA
:10317000B52D480E8827581E0FBE08950FB6F89437
:10318000499059900FBE08955A924A92480E591E7E
:1031900008955A924A92480E8827581E0895480E5C
:1031A0008827581E08950F921F922F92C801D901A7
:1031B000489F80014A9F90014B9F202C499F100DF2
:1031C000211D321D5A9F202C589F100D211D321D8C
:1031D000599F200D311D689F200D311D699F300DB5
:1031E000789F300D2F901F900F9008950E94C21A63
:1031F0000D920020D9F70895369A3699FECF369A67
:103200003699FECF84B195B10895903029F08C9114
:10321000880F9A95E9F78C930895903071F00D918D
:103220001D912D913C91000F111F221F331F9A9564
:10323000D1F73C932E931E930E930895903029F06E
:103240008C9186959A95E9F78C930895903071F05A
:103250000D911D912D913C913695279517950795C8
:103260009A95D1F73C932E931E930E9308953DD0DB
:10327000992711278F2D880F80E8F82A802F881F23
:1032800008F41FEF41F08F57082F07FD04C00032EC
:1032900040F08FEF01C08827982FD82EE82EF82E07
:1032A00009C08FE1801B082FF694E794D794979577
:1032B0000A95D1F7112351F09095D094E094F094B1
:1032C00081E0980F8827D81EE81EF81E0F2DFE2CCF
:1032D000ED2CD92E0895D094E094F09491E0D90E7D
:1032E0009927E91EF91E10950895D190E190F1906B
:1032F0000191089521913191419151910895102F9B
:1033000090E8FF0C001F0927990FF7941078652F9C
:1033100090E8440F551F5927990F4795607800385A
:103320000895FF0C90E89027110F9795F794092FB7
:103330000895102FBD2CDE2CEF2CF02E11234AF413
:10334000B094D094E094F0949FEFB91AD90AE90AA6
:10335000F90A0EE1FF2039F4FE2CED2CDB2CBB2406
:103360000850C2F75EC032F00A95BB0CDD1CEE1CA3
:10337000FF1CF9CF0E948618D4CFDD92ED92FD920A
:103380000C930895502F2D2D3E2D4F2D612F089514
:103390002DEC3CEC4CEC5DE366270FC0A6DFF2DFC2
:1033A000DD24EE2490E8F92E0FE307C0A3DF05C06B
:1033B0002227332740E251E46627552351F10023A9
:1033C00081F19DDF71F11627005850580894050BC4
:1033D00018F407FD03C025C007FD23C046953795A7
:1033E0002795F694E794D79422D0FF202AF0DD0C9D
:1033F000EE1CFF1C015073F09D2D969548F0DD20CA
:103400003AF4EE202AF491E0D90E9927E91EF91E2C
:1034100088CF07C09FE7092FF92A9FEFD92EE92E01
:103420000895DD24EE24FF240027112708959F929C
:103430009924AA24BB2488E1D216E306F40628F0D6
:10344000D21AE30AF40A089401C08894991CAA1CB1
:10345000BB1CDD0CEE1CFF1C8A9571F7D92CEA2CE5
:10346000FB2C9F9008954BDFE1F25038D1F21627E4
:10347000005850580894051F12F418F4CBCF08F0E8
:10348000D0CF0BD0FF202AF0BB0CDD1CEE1CFF1CA4
:1034900048CF0F5F0BF4BECF44CF9F929924AA244C
:1034A000BB24992788E1990CAA1CBB1CDD1CEE1CCF
:1034B000FF1C30F4920EA31EB41ED91EE91EF91E85
:1034C0008A9589F79F90089515DF19DF503829F004
:1034D00090E869270CC00AF045D023CF5FE322278C
:1034E0003327442701C006DF0ADF5038B1F3003824
:1034F00099F3902F951B8BF312F434D0FACF9831B7
:1035000018F0222733274427983028F0232F342F10
:1035100044279850F9CF992329F046953795279558
:103520009A95D9F7912F962742F014D0B0F6F794D8
:10353000E794D7940F5F8BF66DCF10D051F008F45D
:10354000CADEFF2052F2DD0CEE1CFF1C0150CBF74F
:1035500061CF67CFD20EE31EF41E0895D21AE30A9C
:10356000F40A0895DF92EF92FF920F931F93D22EE9
:10357000E32EF42E052F162F6F915F914F913F91FF
:103580002F910895C895319600200895FBDFD02C27
:10359000F9DFE02CF7DFF02CF5DF002D0895F2DFE6
:1035A000202DF0DF302DEEDF402DECDF502D089583
:1035B00007FB00680EF40F7757FB50680EF45F7737
:1035C00007FD02C057FF05C0D216E306F406050743
:1035D00008952D153E054F055007089500240D2828
:1035E0000E280F28002A0020089591E005C092E0DF
:1035F00003C094E001C098E0C5DF0D929A95E1F711
:1036000008952E2E3F2E992781918D3209F09395A2
:103610008823D1F79A95E22DF32D112361F0091734
:1036200018F011F0101B01C0191B28F021F080E2E6
:103630008D931A95E9F780818D3219F48D93319627
:1036400004C0222311F08BE28D93091738F031F07A
:10365000091B21F080E38D930A95E9F781918D9301
:103660008823E1F7332351F0EA2FFB2F319633956E
:103670008E9182933A95E1F78EE28C930895040F30
:10368000151F261F371F0895041B150B260B370B1C
:10369000089504171507260737070895000F111F0F
:1036A000221F331F089500951095209530950F5FC8
:1036B0001F4F2F4F3F4F0895019110810EC0019170
:1036C0001191219130810BC00191108117FF05C02C
:1036D0003FEF2FEF04C0008111272227332737FF48
:1036E00003C0E1DF8DE28D93CF93DF93CF92DF9222
:1036F000EF92AA24BB24CC24DD24EE2440E2CAE0CD
:10370000DD2755E093E38881890F87FD9F7083FD56
:10371000907F891B89935A95A9F7C0DFAA1CBB1C0F
:10372000CC1CDD1CEE1C4A9551F7E894EFE0FF2716
:1037300082910ED0EB30E0F71EF068948A2D0CD009
:1037400088278D93EF90DF90CF90DF91CF910895F0
:10375000982F829501D0892F8F70805D26F080335D
:1037600009F4089568948D9308950027112722275E
:1037700033271DD08A3328F4803318F005D015D0B4
:10378000F9CF0EF490CF089580538F93402F512F8F
:10379000622F732F83DF82DF72DF80DF8F919927A3
:1037A000080F191F291F391F08958D910895E89456
:1037B000FCDF8032E9F38B32D9F38930C9F38D32E3
:1037C00011F46894F2CF089588278D93089581911C
:1037D0008D938823E1F7089594E081918D939A95D4
:1037E000E1F7089509919191992351F08A95D9F7BC
:1037F000319781918D930A9519F08823D1F7089517
:10380000E3CFE199FECFEEBBFFBB3196089591E087
:1038100001C092E07B3751F47FB7F894F2DF8D91CD
:103820008DBBE29AE19A9A95C9F77FBF77270895F1
:1038300091E001C092E0E5DFE09A8DB38D939A9517
:10384000D1F70895FF93881BF9E0001FFA9511F452
:10385000FF910895881F841B18F4840F8894F5CF76
:103860000894F3CF8FEF83959D919923E1F7089505
:10387000689401C0E894AF93BF938D9116F0919135
:1038800003C00E94C21A902D891718F011F48823E2
:10389000A1F7BF91AF910895C4CD27DD0023E2F3D6
:1038A0009DDE19F4B7DD0068089585E05ADCFF0C51
:1038B000001F04830FE70695F79449D0506814DE83
:1038C0005CDD139721E438E743ED5BEBCCDD27E8C3
:1038D00031ED43E15DE337D02EE03CE343EC5DEBBB
:1038E00032D022E83DEA4BE25EE32DD02CEE32E806
:1038F00046E75EEB28D020E931EE49EA5EE323D0CB
:1039000020E83FEE4FEF5EEB1ED024EC3FEF4FE799
:103910005FE319D032DD139784818F5799F02AF431
:10392000D82E0FEFE02EF02E04C0D82EEE24FF2468
:103930000027FFDC28E132E741E35FE394DDDADCD6
:103940003497D2DD1BCCD0DDD5DC34978CCD5FE352
:1039500040E8332722270895A998A898A198A0980D
:103960000895A09AA19803D0A09801D0A19AEF93AE
:10397000FF93E4E0F0E00E944E15FF91EF9108956F
:10398000A09AA19AF4DFA098989BFECFF0DFA198AF
:10399000EECF0894111F01C0110F69F0A09A18F41E
:1039A0000000A19802C0A19A00C0E1DFA098989BF6
:1039B000FECFDDDFF1CFA09AA198D9DFA098989B28
:1039C000FECFE8949999689462F8D1CF089401C029
:1039D0008894331F11E0A09AA198C9DFA098989B02
:1039E000FECFC5DF889499990894111FA0F7A09A7B
:1039F000379510F4A19801C0A19AB9DFA098989BBF
:103A0000FECFB5DF089500000000000000000000B8
:103A1000A0400000803F00008043000040400000C4
:103A200000000000B0410000000000DB8A410000FF
:103A3000001023459B4100000010EE389B41000020
:103A40000000443C9B4100000000000059404260DF
:103A5000653B5053313B000049463B00494600005E
:103A60003B005A5A58543B005A5A5854000050537D
:103A70003B00505300005A5A534D303B00005A5AF5
:103A8000534D0000464100005A5A50413B005A5ADB
:103A9000504100004D4F3B0050433030353B00005B
:083AA00050433030303B0000C0
:00000001FF
